:020000040000FA
:0A0000000000000097EF01F0A5D109
:08001800F2D1076A066EFF0E2B
:100020000626072200D0D8A01200030E056EE60EA9
:1000300002D8F5D7056AFE0F046EE86A055AD8A003
:1000400012000000040600D0F8D7800E1C1A1B50C6
:10005000175C206E11E2206C17501BC017F01B6E4E
:1000600018501CC018F01C6E19501DC019F01D6EE0
:100070001A501EC01AF01E6E1A0E206074D01B5249
:1000800072E01F6A1850226E1C18236E188E1C8E88
:10009000080E205E08E31EC01FF01DC01EF01CC02D
:1000A0001DF01C6AF5D7202607E0D8901C321D32BF
:1000B0001E321F32202EF9D723AE33D01E501A5EC7
:1000C0001D50195A1C50185A07E2D880000E1A56B3
:1000D00019561856800E221A1F6C04E01A06000EDC
:1000E000195A185A040E206E18660DD019C018F04F
:1000F0001AC019F01FC01AF01F6A080E175E29E314
:10010000202EF2D726D018BE08D0D8901F361A3627
:1001100019361836172EF7D71CD01FAE22D01F6AFB
:100120000FD01E501A261D5019221C50182206E30B
:10013000183219321A321F32174A0DD01FAE11D0A1
:100140001A3E0FD0193E0DD0183E0BD0D8801A9011
:10015000EFD7176A02D0218217681A6A196A800ECF
:10016000186E22AE189E1A5012001850166E1C18E7
:10017000236E1750D8A41B503AE017267E0E03E3D7
:10018000175E03E336D0175E31E31AC014F019C0CE
:1001900015F0168E1C8E1A6A196A186A180E226ECD
:1001A00016321532143206E31E501A261D5019223B
:1001B0001C501822183219321A32222EF1D718BECA
:1001C00007D01A3619361836175210E017061634AB
:1001D00016E31A3E14D0193E12D0183E10D0D88023
:1001E000183219321A32173E0AD003D02184176A06
:1001F00002D0218217681A6A196A800E186E23AE1F
:10020000189E1A50120017C022F018501AC018F089
:100210001A6E1A3622321A32216A1A36223602E34E
:100220002184217E06E12180226A1A6A196A186AED
:100230000BD0222803E0D8801A3206D0D8901A3288
:1002400002E1218201D0218621B604D021A20FD063
:1002500021B407D07F0E1A6EFF0E196E186E176E3E
:1002600023D0800E1A6E01D01A6A000EF6D721B084
:10027000FBD7176A9F0E2260EBD77E0E2264F4D75D
:100280009E0E225C07E0D8901A32193218321732CB
:10029000222AF6D721A408D0D880000E1756185667
:1002A00019561A561AAEE0D717501200176E186A70
:1002B000196A1A6A239E0AD0239E1AAE07D0D880E4
:1002C000000E1756185619561A56238E960E226E81
:1002D0001A5209E0080E222618C017F019C018F0AB
:1002E0001AC019F011D019520FE1080E225E1850F1
:1002F00007E1080E225E175002E11A5010D0176A6B
:10030000196E17C018F0176A19BE06D0D8901736A4
:10031000183619362206F8D723AE199E225017C078
:100320001AF0176E195018C019F0186E1200400E0E
:10033000216E4F0EAF6E240EAC6E900EAB6E0001B0
:10034000C69AC00E926E936A946E0F0EC16E070E1F
:10035000B46E6CD0F2A403D0F294827011009EAA05
:1003600019D0060EAB1412E1E2CF25F0E1CF24F054
:10037000262A10EE80F02650E126000EE222AECFB3
:10038000E7FF25C0E2FF24C0E1FF1100AE50AE50F0
:10039000AB98AB8811002650275C14E0272AEACFDF
:1003A00005F0E9CF04F000EE80F02750E926000EBA
:1003B000EA22EF50046E05C0EAFF04C0E9FFD880CE
:1003C000120004D0E868046ED8A012001200266A59
:1003D000276A9D8A9F8AF28EF28C12009D9A00EE07
:1003E00080F0010EF46EF36AF306000EF45AEE6A22
:1003F000F450F310F9E1266A276A9D8A1200F29EF2
:10040000E0CFD5F3D8CFD6F3E8CFD7F3F28E000103
:10041000A192F29ED5C3E0FFD6C3D8FFD7C3E8FFB1
:10042000F28E10009EA8FED7AD6E1200939A8A9AA3
:1004300093968A96949A8B9A93928A92929489949C
:1004400092928992929089909296899692988998A0
:10045000929A899A939E8A9E939C8A9C93988A9852
:1004600093948A9494988B9893908A9094928B9278
:1004700094948B94320E0DEC00F05C6A5B6A5E6AB9
:100480005D6A606A5F6A626A616A646A636A666A10
:10049000656A686A676A6A6A696A6C6A6B6A6E6AC0
:1004A0006D6A706A6F6A726A716A746A736A766A70
:1004B000756A786A776A7A6A796A0101826B836BF6
:1004C000846B856B866B876B886B896B8A6B8B6B98
:1004D0008C6B8D6B8E6B8F6B906B916B346AD26B68
:1004E0000001AEEC11F0CDEC11F0336A326A316AE2
:1004F000306A6DDF73DFCD6AF294F28A870ED56EB3
:10050000B16AA192B368E20EB26E01EE92F0400EB3
:10051000EE68E82EFDD77F687E8E386A376A366AC5
:10052000356A392AE86A39B2010F3AB0010806E1A2
:100530003A70352A000E3622372238222CDF286EF8
:10054000BC0E285C06E3FE0E285CD8A02A6AB8EF31
:100550000BF028AE22D02A6A8B0E285C04E128C05A
:100560002AF02B6816D09B0E285C04E128C02AF0E4
:100570002C680FD0AB0E285C04E128C02AF02E684E
:1005800008D0BB0E285C04E128C02AF00101806974
:100590000001B8EF0BF0B6EF0BF02A5204E1B8EF10
:1005A0000BF0B6EF0BF08B0E2A5CD8A45FD02B2893
:1005B00005E128C02BF0B8EF0BF056D02C0E2B5CC9
:1005C00002E132904ED02D0E2B5C02E1329249D0E6
:1005D0002E0E2B5C02E1329444D02F0E2B5C02E1F4
:1005E00032963FD0300E2B5C02E132983AD0310E79
:1005F0002B5C02E1329A35D0320E2B5C02E1329C48
:1006000030D0330E2B5C02E1329E2BD0340E2B5CAB
:1006100002E1339026D0350E2B5C02E1339221D0DB
:10062000360E2B5C02E133941CD0370E2B5C02E1BA
:10063000339617D0380E2B5C02E1339812D0390E66
:100640002B5C02E1339A0DD03A0E2B5C02E1339C15
:1006500008D03B0E2B5C02E1339E03D02B68B8EF31
:100660000BF02B68B6EF0BF0B6EF0BF09B0E2A5C8D
:10067000D8A4EBEF09F02C2804E128C02CF0EAEF15
:1006800009F028C02DF02D52D8A4D6D02C0E2C5C09
:100690000AE1329030B005D00101956994699369FF
:1006A00092690001C6D02D0E2C5C0AE1329230B264
:1006B00005D0010199699869976996690001B9D0D7
:1006C0002E0E2C5C0AE1329430B405D001019D69F4
:1006D0009C699B699A690001ACD02F0E2C5C0AE1E1
:1006E000329630B605D00101A169A0699F699E6963
:1006F00000019FD0300E2C5C0AE1329830B805D052
:100700000101A569A469A369A269000192D0310E13
:100710002C5C0AE1329A30BA05D00101A969A869B6
:10072000A769A669000185D0320E2C5C0AE1329CD3
:1007300030BC05D00101AD69AC69AB69AA690001A3
:1007400078D0330E2C5C0AE1329E30BE05D0010118
:10075000B169B069AF69AE6900016BD0340E2C5C31
:100760000AE1339031B005D00101B569B469B369CC
:10077000B26900015ED0350E2C5C0AE1339231B2D1
:1007800005D00101B969B869B769B669000151D0EE
:10079000360E2C5C0AE1339431B405D00101BD69F9
:1007A000BC69BB69BA69000144D0370E2C5C0AE110
:1007B000339631B605D00101C169C069BF69BE6910
:1007C000000137D0380E2C5C0AE1339831B805D0DF
:1007D0000101C569C469C369C26900012AD0390E23
:1007E0002C5C0AE1339A31BA05D00101C969C869A4
:1007F000C769C66900011DD03A0E2C5C0AE1339C22
:1008000031BC05D00101CD69CC69CB69CA69000151
:1008100010D03B0E2C5C0AE1339E31BE05D00101A5
:10082000D169D069CF69CE69000103D02C68B8EFD7
:100830000BF02C68B6EF0BF02C0E2C5CD8A459D022
:100840008A8A01EED5F0D8902D34E926000EEA22EE
:10085000EECF3BF0EFCF3CF030803B503524006EC4
:100860003C503620016E000E3720026E000E3820FC
:10087000036E03C095F102C094F101C093F100C072
:1008800092F101018253000131E03280D8903B3473
:100890000101D36F3C34D46F02EED5F0D89082358D
:1008A000E926000EEA22EECF00F0EFCF01F0005073
:1008B000D35D0150D459000105E3D4C15CF0D3C12C
:1008C0005BF012D002EED5F0D89001018235E92616
:1008D000000EEA22EECF00F0EFCF01F0D351005C22
:1008E0005B6ED45101585C6E000101D03290E8EF8C
:1008F00009F02D0E2C5CD8A459D08A8601EED5F0D3
:10090000D8902D34E926000EEA22EECF3DF0EFCF4D
:100910003EF030823D503524006E3E503620016E50
:10092000000E3720026E000E3820036E03C099F1CE
:1009300002C098F101C097F100C096F10101835304
:10094000000131E03282D8903D340101D36F3E3452
:10095000D46F02EED5F0D8908335E926000EEA2256
:10096000EECF00F0EFCF01F00050D35D0150D4592D
:10097000000105E3D4C15EF0D3C15DF012D002EEF8
:10098000D5F0D89001018335E926000EEA22EECF9A
:1009900000F0EFCF01F0D351005C5D6ED4510158EF
:1009A0005E6E000101D03292E8EF09F02E0E2C5C51
:1009B000D8A459D08B8A01EED5F0D8902D34E926F1
:1009C000000EEA22EECF3FF0EFCF40F030843F50F0
:1009D0003524006E40503620016E000E3720026E26
:1009E000000E3820036E03C09DF102C09CF101C0CF
:1009F0009BF100C09AF101018453000131E032847F
:100A0000D8903F340101D36F4034D46F02EED5F05B
:100A1000D8908435E926000EEA22EECF00F0EFCF21
:100A200001F00050D35D0150D459000105E3D4C159
:100A300060F0D3C15FF012D002EED5F0D890010182
:100A40008435E926000EEA22EECF00F0EFCF01F068
:100A5000D351005C5F6ED4510158606E000101D02B
:100A60003294E8EF09F02F0E2C5CD8A459D08A827A
:100A700001EED5F0D8902D34E926000EEA22EECF13
:100A800041F0EFCF42F0308641503524006E4250A5
:100A90003620016E000E3720026E000E3820036EE5
:100AA00003C0A1F102C0A0F101C09FF100C09EF1FE
:100AB00001018553000131E03286D89041340101B3
:100AC000D36F4234D46F02EED5F0D8908535E92645
:100AD000000EEA22EECF00F0EFCF01F00050D35D20
:100AE0000150D459000105E3D4C162F0D3C161F0D3
:100AF00012D002EED5F0D89001018535E926000E1E
:100B0000EA22EECF00F0EFCF01F0D351005C616E2E
:100B1000D4510158626E000101D03296E8EF09F01D
:100B2000300E2C5CD8A459D0898401EED5F0D89031
:100B30002D34E926000EEA22EECF43F0EFCF44F049
:100B4000308843503524006E44503620016E000E2C
:100B50003720026E000E3820036E03C0A5F102C0DC
:100B6000A4F101C0A3F100C0A2F10101865300016C
:100B700031E03288D89043340101D36F4434D46FCC
:100B800002EED5F0D8908635E926000EEA22EECFA7
:100B900000F0EFCF01F00050D35D0150D4590001B7
:100BA00005E3D4C164F0D3C163F012D002EED5F0F6
:100BB000D89001018635E926000EEA22EECF00F03A
:100BC000EFCF01F0D351005C636ED4510158646ED5
:100BD000000101D03298E8EF09F0310E2C5CD8A466
:100BE00059D0898201EED5F0D8902D34E926000E37
:100BF000EA22EECF45F0EFCF46F0308A455035245B
:100C0000006E46503620016E000E3720026E000E38
:100C10003820036E03C0A9F102C0A8F101C0A7F1FA
:100C200000C0A6F101018753000131E0328AD8905B
:100C300045340101D36F4634D46F02EED5F0D8901D
:100C40008735E926000EEA22EECF00F0EFCF01F063
:100C50000050D35D0150D459000105E3D4C166F0C2
:100C6000D3C165F012D002EED5F0D89001018735DE
:100C7000E926000EEA22EECF00F0EFCF01F0D351CB
:100C8000005C656ED4510158666E000101D0329A45
:100C9000E8EF09F0320E2C5CD8A459D0898001EE1F
:100CA000D5F0D8902D34E926000EEA22EECF47F099
:100CB000EFCF48F0308C47503524006E4850362036
:100CC000016E000E3720026E000E3820036E03C046
:100CD000ADF102C0ACF101C0ABF100C0AAF101015D
:100CE0008853000131E0328CD89047340101D36F32
:100CF0004834D46F02EED5F0D8908835E926000E3E
:100D0000EA22EECF00F0EFCF01F00050D35D0150AA
:100D1000D459000105E3D4C168F0D3C167F012D003
:100D200002EED5F0D89001018835E926000EEA22BE
:100D3000EECF00F0EFCF01F0D351005C676ED451DD
:100D40000158686E000101D0329CE8EF09F0330EC3
:100D50002C5CD8A459D0898601EED5F0D8902D34DA
:100D6000E926000EEA22EECF49F0EFCF4AF0308EAE
:100D700049503524006E4A503620016E000E37204F
:100D8000026E000E3820036E03C0B1F102C0B0F154
:100D900001C0AFF100C0AEF101018953000131E0A3
:100DA000328ED89049340101D36F4A34D46F02EEA9
:100DB000D5F0D8908935E926000EEA22EECF00F072
:100DC000EFCF01F00050D35D0150D459000105E38D
:100DD000D4C16AF0D3C169F012D002EED5F0D89038
:100DE00001018935E926000EEA22EECF00F0EFCFAF
:100DF00001F0D351005C696ED45101586A6E000154
:100E000001D0329EE8EF09F0340E2C5CD8A459D002
:100E1000898801EED5F0D8902D34E926000EEA221B
:100E2000EECF4BF0EFCF4CF031804B503524006EBD
:100E30004C503620016E000E3720026E000E382016
:100E4000036E03C0B5F102C0B4F101C0B3F100C03C
:100E5000B2F101018A53000131E03380D8904B3464
:100E60000101D36F4C34D46F02EED5F0D8908A359F
:100E7000E926000EEA22EECF00F0EFCF01F000509D
:100E8000D35D0150D459000105E3D4C16CF0D3C146
:100E90006BF012D002EED5F0D89001018A35E92628
:100EA000000EEA22EECF00F0EFCF01F0D351005C4C
:100EB0006B6ED45101586C6E000101D03390E8EF95
:100EC00009F0350E2C5CD8A459D0898A01EED5F0F2
:100ED000D8902D34E926000EEA22EECF4DF0EFCF68
:100EE0004EF031824D503524006E4E503620016E4A
:100EF000000E3720026E000E3820036E03C0B9F1D9
:100F000002C0B8F101C0B7F100C0B6F101018B53C6
:100F1000000131E03382D8904D340101D36F4E345B
:100F2000D46F02EED5F0D8908B35E926000EEA2278
:100F3000EECF00F0EFCF01F00050D35D0150D45957
:100F4000000105E3D4C16EF0D3C16DF012D002EE02
:100F5000D5F0D89001018B35E926000EEA22EECFBC
:100F600000F0EFCF01F0D351005C6D6ED451015809
:100F70006E6E000101D03392E8EF09F0360E2C5C62
:100F8000D8A458D08A8E01EED5F0D8902D34E92619
:100F9000000EEA22EECF4FF0EFCF50F031844F50E9
:100FA0003524006E50503620016E000E3720026E40
:100FB000000E3820036E03C0BDF102C0BCF101C0B9
:100FC000BBF100C0BAF101018C53000131E0338460
:100FD000D8904F340101D36F5034D46F02EED5F066
:100FE000D8908C35E926000EEA22EECF00F0EFCF44
:100FF00001F00050D35D0150D459000105E3D4C184
:1010000070F0D3C16FF012D002EED5F0D89001018C
:101010008C35E926000EEA22EECF00F0EFCF01F08A
:10102000D351005C6F6ED4510158706E000101D035
:101030003394CED1370E2C5CD8A458D08A8C01EED4
:10104000D5F0D8902D34E926000EEA22EECF51F0EB
:10105000EFCF52F0318651503524006E5250362079
:10106000016E000E3720026E000E3820036E03C0A2
:10107000C1F102C0C0F101C0BFF100C0BEF1010169
:101080008D53000131E03386D89051340101D36F84
:101090005234D46F02EED5F0D8908D35E926000E8B
:1010A000EA22EECF00F0EFCF01F00050D35D015007
:1010B000D459000105E3D4C172F0D3C171F012D04C
:1010C00002EED5F0D89001018D35E926000EEA2216
:1010D000EECF00F0EFCF01F0D351005C716ED45130
:1010E0000158726E000101D0339672D1380E2C5C1B
:1010F000D8A458D08A8801EED5F0D8902D34E926AE
:10110000000EEA22EECF53F0EFCF54F03188535067
:101110003524006E54503620016E000E3720026ECA
:10112000000E3820036E03C0C5F102C0C4F101C037
:10113000C3F100C0C2F101018E53000131E03388D8
:10114000D89053340101D36F5434D46F02EED5F0EC
:10115000D8908E35E926000EEA22EECF00F0EFCFD0
:1011600001F00050D35D0150D459000105E3D4C112
:1011700074F0D3C173F012D002EED5F0D890010113
:101180008E35E926000EEA22EECF00F0EFCF01F017
:10119000D351005C736ED4510158746E000101D0BC
:1011A000339816D1390E2C5CD8A458D08A8401EE1D
:1011B000D5F0D8902D34E926000EEA22EECF55F076
:1011C000EFCF56F0318A55503524006E56503620F8
:1011D000016E000E3720026E000E3820036E03C031
:1011E000C9F102C0C8F101C0C7F100C0C6F10101D8
:1011F0008F53000131E0338AD89055340101D36F09
:101200005634D46F02EED5F0D8908F35E926000E13
:10121000EA22EECF00F0EFCF01F00050D35D015095
:10122000D459000105E3D4C176F0D3C175F012D0D2
:1012300002EED5F0D89001018F35E926000EEA22A2
:10124000EECF00F0EFCF01F0D351005C756ED451BA
:101250000158766E000101D0339ABAD03A0E2C5C58
:10126000D8A458D08B8801EED5F0D8902D34E9263B
:10127000000EEA22EECF57F0EFCF58F0318C5750E6
:101280003524006E58503620016E000E3720026E55
:10129000000E3820036E03C0CDF102C0CCF101C0B6
:1012A000CBF100C0CAF101019053000131E0338C51
:1012B000D89057340101D36F5834D46F02EED5F073
:1012C000D8909035E926000EEA22EECF00F0EFCF5D
:1012D00001F00050D35D0150D459000105E3D4C1A1
:1012E00078F0D3C177F012D002EED5F0D89001019A
:1012F0009035E926000EEA22EECF00F0EFCF01F0A4
:10130000D351005C776ED4510158786E000101D042
:10131000339C5ED03B0E2C5CD8A458D08A8001EE62
:10132000D5F0D8902D34E926000EEA22EECF59F000
:10133000EFCF5AF0318E59503524006E5A50362076
:10134000016E000E3720026E000E3820036E03C0BF
:10135000D1F102C0D0F101C0CFF100C0CEF1010146
:101360009153000131E0338ED89059340101D36F8D
:101370005A34D46F02EED5F0D8909135E926000E9C
:10138000EA22EECF00F0EFCF01F00050D35D015024
:10139000D459000105E3D4C17AF0D3C179F012D059
:1013A00002EED5F0D89001019135E926000EEA222F
:1013B000EECF00F0EFCF01F0D351005C796ED45145
:1013C00001587A6E000101D0339E02D02C68D0D132
:1013D0002C68CCD1CBD1AB0E2A5CD8A4B8D12E28A6
:1013E00004E128C02EF0C4D1B1D12C0E2E5C18E13E
:1013F00028C082F10101825300010EE002EED5F017
:10140000D89001018235E926000EEA22EECF5BF08A
:10141000EFCF5CF0000103D05C6A5B6A329094D13C
:101420002D0E2E5C18E128C083F1010183530001C9
:101430000EE002EED5F0D89001018335E926000ECA
:10144000EA22EECF5DF0EFCF5EF0000103D05E6ADE
:101450005D6A329279D12E0E2E5C18E128C084F19B
:101460000101845300010EE002EED5F0D890010195
:101470008435E926000EEA22EECF5FF0EFCF60F070
:10148000000103D0606A5F6A32945ED12F0E2E5C39
:1014900018E128C085F10101855300010EE002EE3C
:1014A000D5F0D89001018535E926000EEA22EECF6D
:1014B00061F0EFCF62F0000103D0626A616A329698
:1014C00043D1300E2E5C18E128C086F1010186530D
:1014D00000010EE002EED5F0D89001018635E92634
:1014E000000EEA22EECF63F0EFCF64F0000103D0EC
:1014F000646A636A329828D1310E2E5C18E128C0E4
:1015000087F10101875300010EE002EED5F0D8907B
:1015100001018735E926000EEA22EECF65F0EFCF14
:1015200066F0000103D0666A656A329A0DD1320E08
:101530002E5C18E128C088F10101885300010EE0FB
:1015400002EED5F0D89001018835E926000EEA2296
:10155000EECF67F0EFCF68F0000103D0686A676AEA
:10156000329CF2D0330E2E5C18E128C089F10101C3
:10157000895300010EE002EED5F0D89001018935C3
:10158000E926000EEA22EECF69F0EFCF6AF0000103
:1015900003D06A6A696A329ED7D0340E2E5C18E195
:1015A00028C08AF101018A5300010EE002EED5F055
:1015B000D89001018A35E926000EEA22EECF6BF0C1
:1015C000EFCF6CF0000103D06C6A6B6A3390BCD033
:1015D000350E2E5C18E128C08BF101018B53000100
:1015E0000EE002EED5F0D89001018B35E926000E11
:1015F000EA22EECF6DF0EFCF6EF0000103D06E6AFD
:101600006D6A3392A1D0360E2E5C18E128C08CF1A1
:1016100001018C5300010EE002EED5F0D8900101DB
:101620008C35E926000EEA22EECF6FF0EFCF70F096
:10163000000103D0706A6F6A339486D0370E2E5C37
:1016400018E128C08DF101018D5300010EE002EE7A
:10165000D5F0D89001018D35E926000EEA22EECFB3
:1016600071F0EFCF72F0000103D0726A716A3396A5
:101670006BD0380E2E5C18E128C08EF101018E531C
:1016800000010EE002EED5F0D89001018E35E9267A
:10169000000EEA22EECF73F0EFCF74F0000103D01A
:1016A000746A736A339850D0390E2E5C18E128C0E2
:1016B0008FF101018F5300010EE002EED5F0D890BA
:1016C00001018F35E926000EEA22EECF75F0EFCF4B
:1016D00076F0000103D0766A756A339A35D03A0EF7
:1016E0002E5C18E128C090F10101905300010EE03A
:1016F00002EED5F0D89001019035E926000EEA22DD
:10170000EECF77F0EFCF78F0000103D0786A776AF8
:10171000339C1AD03B0E2E5C17E128C091F10101D9
:10172000915300010EE002EED5F0D8900101913501
:10173000E926000EEA22EECF79F0EFCF7AF0000131
:1017400003D07A6A796A339E2E6812D00FD0BB0E0E
:101750002A5C0CE101018029000104E128C080F12C
:1017600007D004D028C081F113EC10F0D9EC0FF0B1
:10177000100E7F5CD8B0D0EF0FF07B50355C7C5002
:1017800036587D5037587E503858D8A0AFEF0FF0FC
:101790007E8E7F523CE132B009D08A9A30900101AE
:1017A000956994699369926900012FD030A017D090
:1017B0008A9A5B503524006E5C503620016E000E14
:1017C0003720026E000E3820036E03C095F102C070
:1017D00094F101C093F100C092F1309016D08A8A42
:1017E0003B503524006E3C503620016E000E3720F1
:1017F000026E000E3820036E03C095F102C094F112
:1018000001C093F100C092F13080AEEF0FF0010EF5
:101810007F5C3CE132B209D08A963092010199692D
:1018200098699769966900012FD030A217D08A96DF
:101830005D503524006E5E503620016E000E37205C
:10184000026E000E3820036E03C099F102C098F1B9
:1018500001C097F100C096F1309216D08A863D50B3
:101860003524006E3E503620016E000E3720026E89
:10187000000E3820036E03C099F102C098F101C038
:1018800097F100C096F13082AEEF0FF0020E7F5C50
:101890003CE132B409D08B9A309401019D699C6976
:1018A0009B699A6900012FD030A417D08B9A5F50A2
:1018B0003524006E60503620016E000E3720026E17
:1018C000000E3820036E03C09DF102C09CF101C0E0
:1018D0009BF100C09AF1309416D08B8A3F5035248A
:1018E000006E40503620016E000E3720026E000E52
:1018F0003820036E03C09DF102C09CF101C09BF132
:1019000000C09AF13084AEEF0FF0030E7F5C3CE133
:1019100032B609D08A9230960101A169A0699F6907
:101920009E6900012FD030A617D08A9261503524CD
:10193000006E62503620016E000E3720026E000EDF
:101940003820036E03C0A1F102C0A0F101C09FF1D5
:1019500000C09EF1309616D08A8241503524006E28
:1019600042503620016E000E3720026E000E3820E5
:10197000036E03C0A1F102C0A0F101C09FF100C03D
:101980009EF13086AEEF0FF0040E7F5C3CE132B882
:1019900009D0899430980101A569A469A369A26955
:1019A00000012FD030A817D0899463503524006EE1
:1019B00064503620016E000E3720026E000E382073
:1019C000036E03C0A5F102C0A4F101C0A3F100C0E1
:1019D000A2F1309816D0898443503524006E4450CB
:1019E0003620016E000E3720026E000E3820036E86
:1019F00003C0A5F102C0A4F101C0A3F100C0A2F18F
:101A00003088AEEF0FF0050E7F5C3CE132BA09D0B2
:101A10008992309A0101A969A869A769A66900019C
:101A20002FD030AA17D0899265503524006E6650A9
:101A30003620016E000E3720026E000E3820036E35
:101A400003C0A9F102C0A8F101C0A7F100C0A6F12E
:101A5000309A16D0898245503524006E4650362083
:101A6000016E000E3720026E000E3820036E03C098
:101A7000A9F102C0A8F101C0A7F100C0A6F1308A07
:101A8000AEEF0FF0060E7F5C3CE132BC09D08990CE
:101A9000309C0101AD69AC69AB69AA6900012FD026
:101AA00030AC17D0899067503524006E68503620CE
:101AB000016E000E3720026E000E3820036E03C048
:101AC000ADF102C0ACF101C0ABF100C0AAF1309C95
:101AD00016D0898047503524006E48503620016E5C
:101AE000000E3720026E000E3820036E03C0ADF1E9
:101AF00002C0ACF101C0ABF100C0AAF1308CAEEF76
:101B00000FF0070E7F5C3BE132BE09D08996309E14
:101B10000101B169B069AF69AE6900012FD030AE83
:101B200017D0899669503524006E6A503620016EB0
:101B3000000E3720026E000E3820036E03C0B1F194
:101B400002C0B0F101C0AFF100C0AEF1309E16D0BE
:101B5000898649503524006E4A503620016E000EA9
:101B60003720026E000E3820036E03C0B1F102C0B0
:101B7000B0F101C0AFF100C0AEF1308EEFD1080E70
:101B80007F5C3BE133B009D0899831900101B569A0
:101B9000B469B369B26900012FD031A017D0899818
:101BA0006B503524006E6C503620016E000E3720CD
:101BB000026E000E3820036E03C0B5F102C0B4F10E
:101BC00001C0B3F100C0B2F1319016D089884B50FA
:101BD0003524006E4C503620016E000E3720026E08
:101BE000000E3820036E03C0B5F102C0B4F101C08D
:101BF000B3F100C0B2F13180B1D1090E7F5C3BE19D
:101C000033B209D0899A31920101B969B869B769CB
:101C1000B66900012FD031A217D0899A6D503524B2
:101C2000006E6E503620016E000E3720026E000EE0
:101C30003820036E03C0B9F102C0B8F101C0B7F19A
:101C400000C0B6F1319216D0898A4D503524006E0D
:101C50004E503620016E000E3720026E000E3820E6
:101C6000036E03C0B9F102C0B8F101C0B7F100C002
:101C7000B6F1318273D10A0E7F5C3BE133B409D0F7
:101C80008A9E31940101BD69BC69BB69BA690001D2
:101C90002FD031A417D08A9E6F503524006E70501B
:101CA0003620016E000E3720026E000E3820036EC3
:101CB00003C0BDF102C0BCF101C0BBF100C0BAF16C
:101CC000319416D08A8E4F503524006E50503620F5
:101CD000016E000E3720026E000E3820036E03C026
:101CE000BDF102C0BCF101C0BBF100C0BAF131844A
:101CF00035D10B0E7F5C3BE133B609D08A9C31961F
:101D00000101C169C069BF69BE6900012FD031A658
:101D100017D08A9C71503524006E72503620016EA7
:101D2000000E3720026E000E3820036E03C0C1F192
:101D300002C0C0F101C0BFF100C0BEF1319616D0A3
:101D40008A8C51503524006E52503620016E000EA0
:101D50003720026E000E3820036E03C0C1F102C0AE
:101D6000C0F101C0BFF100C0BEF13186F7D00C0E4A
:101D70007F5C3BE133B809D08A9831980101C5698D
:101D8000C469C369C26900012FD031A817D08A98ED
:101D900073503524006E74503620016E000E3720CB
:101DA000026E000E3820036E03C0C5F102C0C4F1FC
:101DB00001C0C3F100C0C2F1319816D08A885350D7
:101DC0003524006E54503620016E000E3720026E0E
:101DD000000E3820036E03C0C5F102C0C4F101C07B
:101DE000C3F100C0C2F13188B9D00D0E7F5C3BE178
:101DF00033BA09D08A94319A0101C969C869C7699F
:101E0000C66900012FD031AA17D08A9475503524A5
:101E1000006E76503620016E000E3720026E000EE6
:101E20003820036E03C0C9F102C0C8F101C0C7F178
:101E300000C0C6F1319A16D08A8455503524006E00
:101E400056503620016E000E3720026E000E3820EC
:101E5000036E03C0C9F102C0C8F101C0C7F100C0E0
:101E6000C6F1318A7BD00E0E7F5C3BE133BC09D0DA
:101E70008B98319C0101CD69CC69CB69CA6900019D
:101E80002FD031AC17D08B9877503524006E785016
:101E90003620016E000E3720026E000E3820036ED1
:101EA00003C0CDF102C0CCF101C0CBF100C0CAF13A
:101EB000319C16D08B8857503524006E58503620F0
:101EC000016E000E3720026E000E3820036E03C034
:101ED000CDF102C0CCF101C0CBF100C0CAF1318C10
:101EE0003DD00F0E7F5C3AE133BE09D08A90319E1F
:101EF0000101D169D069CF69CE6900012FD031AE1F
:101F000017D08A9079503524006E7A503620016EB1
:101F1000000E3720026E000E3820036E03C0D1F190
:101F200002C0D0F101C0CFF100C0CEF1319E16D079
:101F30008A8059503524006E5A503620016E000EAA
:101F40003720026E000E3820036E03C0D1F102C0AC
:101F5000D0F101C0CFF100C0CEF1318E2AD838AE19
:101F60001ED0386A376A366A356A316A306A336A2F
:101F7000326A01EE92F0400EEE68E82EFDD78A9AA2
:101F80008A968B9A8A92899489928990899689985F
:101F9000899A8A9E8A9C8A988A948B988A9006D07D
:101FA00038AE04D0386A376A366A356A827691EF7D
:101FB00002F07F687E8E296A100E295C33E2D89089
:101FC0002934E96EEA6AEA36E936EA36920EE926FB
:101FD000010EEA22EFCF00F0ECCF01F0ECCF02F0DF
:101FE000ECCF03F07B50005C7C5001587D500258D0
:101FF0007E50035815E2D8902934E96EEA6AEA3631
:10200000E936EA36920EE926010EEA22EFCF7BF09E
:10201000ECCF7CF0ECCF7DF0ECCF7EF029C07FF0F0
:10202000292ACAE312001E0E0101805D0001D8A416
:102030000CD101018153000135E1336A326A5C6AD7
:102040005B6A0101826B5E6A5D6A836B606A5F6ACC
:10205000846B626A616A856B646A636A866B666AAE
:10206000656A876B686A676A886B6A6A696A896B7E
:102070006C6A6B6A8A6B6E6A6D6A8B6B706A6F6A68
:102080008C6B726A716A8D6B746A736A8E6B766A16
:10209000756A8F6B786A776A906B7A6A796A916BE6
:1020A0000001D1D081C182F102EED5F0D8900101BA
:1020B0008135E926000EEA22EECF5BF0EFCF5CF02F
:1020C00081C183F102EED5F0D8908135E926000E6A
:1020D000EA22EECF5DF0EFCF5EF081C184F102EE37
:1020E000D5F0D8908135E926000EEA22EECF5FF0D8
:1020F000EFCF60F081C185F102EED5F0D890813547
:10210000E926000EEA22EECF61F0EFCF62F081C146
:1021100086F102EED5F0D8908135E926000EEA224C
:10212000EECF63F0EFCF64F081C187F102EED5F01E
:10213000D8908135E926000EEA22EECF65F0EFCF88
:1021400066F081C188F102EED5F0D8908135E9269C
:10215000000EEA22EECF67F0EFCF68F081C189F17F
:1021600002EED5F0D8908135E926000EEA22EECFB6
:1021700069F0EFCF6AF081C18AF102EED5F0D89014
:102180008135E926000EEA22EECF6BF0EFCF6CF03E
:1021900081C18BF102EED5F0D8908135E926000E91
:1021A000EA22EECF6DF0EFCF6EF081C18CF102EE3E
:1021B000D5F0D8908135E926000EEA22EECF6FF0F7
:1021C000EFCF70F081C18DF102EED5F0D89081355E
:1021D000E926000EEA22EECF71F0EFCF72F081C156
:1021E0008EF102EED5F0D8908135E926000EEA2274
:1021F000EECF73F0EFCF74F081C18FF102EED5F026
:10220000D8908135E926000EEA22EECF75F0EFCFA7
:1022100076F081C190F102EED5F0D8908135E926B3
:10222000000EEA22EECF77F0EFCF78F081C191F186
:1022300002EED5F0D8908135E926000EEA22EECFE5
:1022400079F0EFCF7AF0000185D0420E0101805D78
:102250000001D8A45BD0010181530001D8A454D05F
:10226000316A306A336A326A01EE92F0400EEE68EB
:10227000E82EFDD77F688A9A8A968B9A8A928994EB
:102280008992899089968998899A8A9E8A9C8A9847
:102290008A948B988A905C6A5B6A5E6A5D6A606AFF
:1022A0005F6A626A616A646A636A666A656A686AC2
:1022B000676A6A6A696A6C6A6B6A6E6A6D6A706A72
:1022C0006F6A726A716A746A736A766A756A786A22
:1022D000776A7A6A796A0101826B836B846B856B9A
:1022E000866B876B886B896B8A6B8B6B8C6B8D6B4A
:1022F0008E6B8F6B906B916B346AD26B386A376AD6
:10230000366A356A000101D0346824D07B0E0101A1
:10231000805D00011FE1316A306A336A326A8A9A4D
:102320008A968B9A8A9289948992899089968998BB
:10233000899A8A9E8A9C8A988A948B988A90386A0D
:10234000376A366A356A01EE92F0400EEE68E82E82
:10235000FDD77F680101806900011200296A800EA3
:10236000295C1AE22950D00DF3CF08F0F4CF09F020
:1023700009260850FF08006EFF0E0954016E02EE98
:10238000D5F0D8902934E926000EEA2200C0EEFFED
:1023900001C0EFFF292AE3E312000101D66B400ED2
:1023A000D56F010E296E0001800E295CD8B06FD068
:1023B0000B6A0A6A180E096E850E086EEC0E0F6E17
:1023C000510E0E6E530E0D6E840E0C6E295056EC8F
:1023D00001F01AC013F019C012F018C011F017C0A4
:1023E00010F01E6A1D6A1C6A7F0E1B6E13C01AF065
:1023F00012C019F011C018F010C017F025EC00F051
:102400001AC013F019C012F018C011F017C010F064
:102410000FC01EF00EC01DF00DC01CF00CC01BF054
:1024200013C01AF012C019F011C018F010C017F044
:10243000B5EC00F01AC00FF019C00EF018C00DF086
:1024400017C00CF00BC01EF00AC01DF009C01CF034
:1024500008C01BF00FC01AF00EC019F00DC018F024
:102460000CC017F027EC00F003EC01F0006E18C070
:1024700001F001EED5F0D8902934E926000EEA22C9
:1024800000C0EEFF01C0EFFF292AD8A08CD71200B0
:02249000FFD774
:020000040030CA
:0300010006170ED1
:020005008580F4
:060008000FC00FE00F40E5
:00000001FF
